:0400000080316328C0
:1000080080310B1D4E28273020009500D208031D93
:100018000F2821009D14FD0A10307D020318FD01F0
:10002800200041087D0203181B280D141C280D1000
:1000380042087D02031822288D1423288D104308B6
:100048007D02031829280D152A280D1144087D0260
:10005800031830288D1531288D1145087D020318A5
:1000680037280D1638280D1246087D0203183E2839
:100078008D163F288D1247087D02031845280D1755
:1000880046280D1348087D0203184C288D174D2863
:100098008D130B112000111F09005308A03E860084
:1000A800870121001C0881002000D30A5308123A56
:1000B800031D6128D301D201D20A11130900880156
:1000C80080316628FD0120308400003085003430FE
:1000D800833121238031A030840000308500123024
:1000E8008331212380310130DE00DF0020009D288C
:1000F800F2014030DE218031F301F30A0830F200CA
:100108007208730203188D288030F0218031F203C1
:1001180084287308F200F20803199728FF30F021A9
:100128008031F2038F28F30A09307302031808009C
:10013800822821009917191799161916991129302B
:10014800FB006E30FA009830F900F90BA928FA0B79
:10015800A928FB0BA928B0288B0121009101920145
:100168002000910192018C018D0122008C018D01EA
:10017800103023008C008D01303021008C008D015F
:10018800950124008C1621009513200098019C01EC
:10019800250093019A01240095010B1720302100B6
:1001A8009E0011309D001117200011132100151118
:1001B80095101510951195120B118B16AE218031E3
:1001C8007C2080318B17200052080319E72804226D
:1001D8008031D2018C1AF928DE0A04305E02031C31
:1001E800F728DE01DE0A5E08DF008C1EF928DF0B27
:1001F800E7285E08DF00FC01FC0A7C08403E860018
:1002080087017C08493E84008501000801027C08BA
:1002180003181629403E86007C08493E84000008E1
:1002280081007C08493E860087017C08403E8400A6
:100238008501000801027C0803182629403E860033
:1002480081037C08403E86008701103001027C084B
:10025800031C3329403E86000F3081007C08403E55
:1002680086008701083001027C08031C5629203EBD
:1002780086007C08403E840085010008F83E810025
:100288007C08203E8600083001027C08031C5129A6
:10029800203E8600073081007C08303E86008701BA
:1002A80007306329203E86008701203081007C08C2
:1002B800303E86007C08403E8400850100088100AD
:1002C8007C08203E860087018108031D75297C086B
:1002D800203E86007C08203E8400850100080838FE
:1002E80081007C08303E860087018108031D86292D
:1002F8007C08303E86007C08303E8400850100087A
:1003080008388100FC0A09307C02031C012980306E
:10031800DE218031FC01FC0A7C08203E8600870132
:100328000108F0218031FC0A09307C02031C902965
:10033800C030DE218031FC01FC0A7C08303E86009A
:1003480087010108F0218031FC0A09307C0203187A
:10035800E728A1299C30F300D730F200F20BB2292C
:10036800F30BB229023022008C000C138C178C136B
:100378003430F300F130F200F20BC029F30BC0293E
:10038800C5292B30DE2180311330DE2180310C303D
:10039800DE2180310430DE2180310130DE218031E0
:1003A8001530F300C630F200F20BD829F30BD82928
:1003B80064000800F100710E0F3922008C008C17C0
:1003C8008C1371080F398C008C178C136A30F0006D
:1003D800F00BEC2964000800F100710E0F392200BF
:1003E8008C000C178C178C1371080F398C000C17A4
:1003F8008C178C136A30F000F00B002A6400080098
:10040800DA01DB01DC01DD01D401D501D801D90114
:100418005408C33E840085300318013E8500000857
:10042800D600D701D635D70DD40A0319D50A5908ED
:10043800A03E860087010108F000F101013056074F
:1004480084008430573D85000008F200F301F21B58
:10045800F303B42280317008DC027108DD3B5908CF
:10046800A03E860087010108F000F1015B305607C5
:1004780084008430573D85000008F200F301F21B28
:10048800F303B42280317008DA077108DB3DD90A1A
:1004980012305902031C0C2A7F30F000F1015D086C
:1004A800F3005C08F200C92280317108DD00700891
:1004B800DC007F30F000F1015B08F3005A08F2001D
:1004C800C92280317108DB007008DA00DD1F792A43
:1004D800FF30F000F1005D08F3005C08F200B42280
:1004E80080317108DD007008DC00DB1F882AFF30CE
:1004F800F000F1005B08F3005A08F200B4228031E2
:100508007108DB007008DA005808493E8600870148
:100518000430F000F1015A085C07F2005B085D3D09
:10052800F300C922803170088100D80A09305802C6
:10053800031C0B2A4A08F800F836F8367808CA006F
:100548000330F0004B080923CB004E35CE004F3561
:10055800CF005035D000510809075107D1000800D5
:10056800F401F501701CBC2A7208F4077308F53D04
:10057800F235F30DF136F00C71087004031DB62A3C
:100588007508F1007408F0000800F501F11FD32A7E
:10059800F009F109F00A0319F10AF501F50AF31F48
:1005A800DC2AF209F309F20A0319F30A0130F50605
:1005B800F601F701710870040319FC2AF401F40A22
:1005C800F11BE92AF035F10DE32AF635F70D71082C
:1005D8007302031DF12A70087202031CF82A7008BE
:1005E800F2027108F33B7614F136F00CF40BE92AA9
:1005F80075080319042BF609F709F60A0319F70A0F
:100608007708F1007608F0000800F100F30170089F
:1006180003191F2BF201F20AF01B142BF0350F2BD4
:10062800F33570087102031C1C2B7008F102731457
:10063800F036F20B142B73080800640080010131B6
:06064800890B222B003497
:100800000034003402340434073409340B340D341A
:100810000F3412341434163418341A341D341F347F
:10082000213423342534273429342B342E343034E6
:1008300032343434363438343A343C343E34403450
:10084000413443344534473449344B344C344E34CA
:100850005034523453345534573458345A345B344A
:100860005D345E34603461346334643465346734D9
:10087000683469346B346C346D346E346F34703476
:100880007134723473347434753476347734773425
:100890007834793479347A347B347B347C347C34E6
:1008A0007D347D347D347E347E347E347F347F34B9
:1008B0007F347F347F347F347F347F347F347F34A0
:1008C0007F347E347E347E347D347D347D347C349C
:1008D0007C347B347B347A347934793478347734AB
:1008E00077347634753474347334723471347034CC
:1008F0006F346E346D346C346B34693468346734FF
:10090000653464346334613460345E345D345B3444
:100910005A345834573455345334523450344E3496
:100920004C344B34493447344534433441344034F7
:100930003E343C343A34383436343434323430345F
:100940002E342B34293427342534233421341F34D6
:100950001D341A3418341634143412340F340D3450
:100960000B3409340734043402340034FE34FC34CC
:10097000F934F734F534F334F134EE34EC34EA344A
:10098000E834E634E334E134DF34DD34DB34D934C5
:10099000D734D534D234D034CE34CC34CA34C8343D
:1009A000C634C434C234C134BF34BD34BB34B934AA
:1009B000B734B534B434B234B034AE34AD34AB340F
:1009C000A934A834A634A534A334A234A0349F3467
:1009D0009D349C349B3499349834973495349434B2
:1009E00093349234913490348F348E348D348C34EB
:1009F0008B348A3489348934883487348734863414
:100A00008534853484348434833483348334823429
:100A1000823482348134813481348134813481342C
:100A2000813481348134813481348234823482341B
:100A300083348334833484348434853485348634F5
:100A4000873487348834893489348A348B348C34BD
:100A50008D348E348F349034913492349334943472
:100A600095349734983499349B349C349D349F3416
:100A7000A034A234A334A534A634A834A934AB34AA
:100A8000AD34AE34B034B234B434B534B734B93430
:100A9000BB34BD34BF34C034C234C434C634C834AB
:100AA000CA34CC34CE34D034D234D534D734D9341B
:100AB000DB34DD34DF34E134E334E634E834EA3483
:100AC000EC34EE34F134F334F534F734F934FC34E7
:100AD000FE34003402340434073409340B340D344A
:100AE0000F3412341434163418341A341D341F34AD
:100AF000213423342534273429342B342E34303414
:100B000032343434363438343A343C343E343F347E
:100B1000413443344534473449344B344C344E34F7
:100B20005034523453345534573458345A345B3477
:100B30005D345E3460346134633464346534673406
:100B4000683469346B346C346D346E346F347034A3
:100B50007134723473347434753476347734773452
:100B60007834793479347A347B347B347C347C3413
:100B70007D347D347D347E347E347E347F347F34E6
:100B80007F347F347F340034003400340034003448
:100B900000340034003400340034003400340034B5
:100BA0000034003400340034003400340A34143487
:100BB0001E34283432343C34463450345A3464348D
:100BC0006E34783482348C349634A034AA340034B1
:100BD000143428343C345034643478348C34A034A5
:100BE0000034143428343C345034643478348C3435
:100BF000A03400341E343C345A34783496340034F3
:100C00001E343C345A347834963400341E343C3428
:100C10005A34783496340034283450347834A0343C
:100C200014343C3464348C340034283450347834F4
:100C3000A03414343C3464348C340034323464349E
:100C40009634143446347834AA3428345A348C34E4
:100C50000A343C346E34A0341E34503482340034B0
:100C60003C34783400343C34783400343C347834C8
:100C700000343C34783400343C34783400343C3430
:100C80007834003446348C341E346434AA343C3412
:100C9000823414345A34A034323478340A34503420
:100CA000963428346E3400345034A0343C348C34C0
:100CB000283478341434643400345034A0343C3450
:0A0CC0008C34283478341434643482
:020000040001F9
:04000E00A4E9FF1C46
:00000001FF
